:100000009BC00000B5C00000B3C00000B1C000003C
:10001000AFC00000ADC00000ABC00000A9C0000030
:10002000A7C00000A5C0000003C60000CCC60000A9
:100030009FC000009DC000009BC0000099C0000050
:1000400097C0000095C0000093C0000091C0000060
:100050008FC000008DC000008BC0000089C0000070
:1000600087C0000085C0000083C0000081C0000080
:100070007FC000007DC000007BC0000079C0000090
:1000800077C0000075C0000073C0000071C00000A0
:100090006FC000006DC000006BC0000069C00000B0
:1000A00067C0000065C0000063C000001C034C0076
:1000B000550046004100200043004400430020005A
:1000C000440065006D006F000000180344006500E7
:1000D00061006E002000430061006D006500720049
:1000E000610000000403090409023E00020100C08F
:1000F000320904000001020201000524001001047D
:100100002402060524060001070582030800FF09F2
:10011000040100020A0000000705040210000507A0
:100120000583021000051201100102000008EB0314
:10013000442001000102DC0111241FBECFEFD5E0F5
:10014000DEBFCDBF11E0A0E0B1E0ECE3FFE102C013
:1001500005900D92A832B107D9F721E0A8E2B1E0ED
:1001600001C01D92A434B207E1F756D10C949C0F44
:1001700047CFAF92BF92DF92EF92FF920F931F9300
:10018000CF93DF935A01DA011D921C92FB01118279
:100190001082EC0120E030E0A1E0B0E0E0E0F0E02F
:1001A0004AE0D42E088119810A30110589F10D32F7
:1001B000110591F00032110589F4A29F8001A39FDF
:1001C000100DB29F100D1124DB010D931C9320E044
:1001D00030E0A1E0B0E002C0AFEFBFEF08811981CD
:1001E000780140E3E41AF1085AE0E516F10450F40E
:1001F000A901D49E9001D59E300D1124200F311FEE
:1002000020533109199219923196E431F10551F6D2
:10021000A29FB001A39F700DB29F700D1124D50154
:100220006D937C93EE0FFF1FE80FF91F1182108270
:10023000DF91CF911F910F91FF90EF90DF90BF90D2
:10024000AF900895CF92DF92EF92FF92CF93DF931A
:1002500089E080937C0080E280937B0085E8809336
:100260007A00CAE0D0E0C12CD12C760180917A00CE
:10027000806480937A0080917A0086FDFCCF609143
:1002800078007091790080E090E00E944B0B20E0B4
:1002900030E040E251E40E94B20A9B01AC01C70188
:1002A000B6010E94370A6B017C0121972097F1F675
:1002B0000E949B0A0E941A0BCB01DF91CF91FF9005
:1002C000EF90DF90CF900895CF92DF92EF92FF9260
:1002D000CF93DF938CE080937C0080E280937B005F
:1002E00085E880937A00CAE0D0E0C12CD12C760159
:1002F00080917A00806480937A0080917A0086FDF4
:10030000FCCF609178007091790080E090E00E94CD
:100310004B0B20E030E040E251E40E94B20A9B0126
:10032000AC01C701B6010E94370A6B017C0121971D
:100330002097F1F60E949B0A0E941A0BCB01DF91D5
:10034000CF91FF90EF90DF90CF9008958F929F9282
:10035000AF92BF92CF92DF92EF92FF9249015A0182
:1003600020E030E044E353E40E94B20A20E030E0B1
:100370004AEF54E40E94410C20E030E04AEF53E49D
:100380000E94370A0E949B0A6B017C0120E030E04A
:1003900044E353E4C501B4010E94B20A20E030E016
:1003A0004AEF54E40E94410C20E030E04AEF53E46D
:1003B0000E94370A0E949B0A4B015C01C701B601EB
:1003C0000E941A0B7093890060938800C501B401E4
:1003D0000E941A0B70938B0060938A00FF90EF903D
:1003E000DF90CF90BF90AF909F908F90089584B78B
:1003F000877F84BF88E10FB6F894809360001092E5
:1004000060000FBE90E080E80FB6F8948093610022
:10041000909361000FBEEFC3CF93DF93CDB7DEB7EC
:10042000E8970FB6F894DEBF0FBECDBF2D98259A82
:100430002E98269A80EA8093800082E18093810042
:1004400080E29EE49093870080938600809880B33A
:100450008C7F80BB80B3807E80BB80B3807C80BB80
:100460001CA61BA61AA619A6FE01319688E2DF017A
:100470001D928A95E9F7BBDF69E271E080E091E0C7
:1004800031D77894812C912CF2E0AF2EF3E4BF2E7B
:1004900075016401AAE04A2EA7ED5A2EA3E26A2E46
:1004A000ACE37A2E4DA65EA66FA678AA212C312C3D
:1004B00080E091E0D9D68C01C5DE9EAB8DAB04DF28
:1004C00098AF8FAB6DA97EA9605C7340882777FDDC
:1004D0008095982F0E944D0B69AB7AAB8BAB9CAB90
:1004E0009F7720E030E040E451E40E943D0C181674
:1004F000D4F5ADA9BEA9A13CB3404CF02AE037ED3C
:1005000043E25CE369A97AA98BA99CA908C029A93F
:100510003AA94BA95CA96DA57EA58FA598A90E94B3
:10052000410C9B01AC01C701B601A0D76B017C0156
:1005300020E030E044E353E40E94AE0A87FF0DC0A0
:1005400020E030E0A901C701B6010E943D0C181659
:1005500054F0C12CD12C760106C0C12CD12CE4E37F
:10056000EE2EE3E4FE2E6FA978AD6D547109882755
:1005700077FD8095982F0E944D0B69AB7AAB8BABC2
:100580009CAB9F7720E030E040EC50E40E943D0CB3
:100590001816D4F58FA998AD8E3491054CF02AE049
:1005A00037ED43EA5CE369A97AA98BA99CA909C044
:1005B000A3019201C301B2015AD729A93AA94BA9B3
:1005C0005CA90E94410C9B01AC01C501B4014FD74D
:1005D0004B015C0120E030E044E353E4BFD787FFE8
:1005E0000DC020E030E0A901C501B4010E943D0C1E
:1005F000181654F0812C912C540106C0812C912C9A
:1006000074E3A72E73E4B72EA5019401C701B601C8
:100610009DDE17FDEAC0C1010196F101EE0FFF1F3B
:10062000A1E0B0E0AC0FBD1FEA0FFB1F11830083F8
:100630000A30110509F0D8C0AE01475D5F4FBE0119
:10064000655D7F4FCD0195DD6BA47CA46627772780
:1006500066197709882777FD8095982F0E944D0BA2
:100660002B018C012FE530E749E850E377D787FF6E
:1006700005C03FE520E709E810E302C0342D252D31
:10068000632F722FC8010E94A80C9B01AC0167E880
:1006900079EA88E49CE366D76DA77EA78FA798AB1D
:1006A0002AE037ED43E25CE359D787FF0FC020E033
:1006B00030E0A9016DA57EA58FA598A94FD787FF2A
:1006C0000DC01DA61EA61FA618AA08C08AE097ED99
:1006D000A3E2BCE38DA79EA7AFA7B8AB94ED6916C4
:1006E0009EEF790624F41DA61EA61FA618AA09A52A
:1006F0001AA566277727601B710B882777FD8095E1
:10070000982FCBD72B013C012FE530E749E850E388
:1007100025D787FF05C05FE540E739E820E304C03F
:10072000542D452D362D272D652F742F832F922F75
:100730000E94A80C9B01AC0167E879EA88E49CE37D
:1007400011D72B013C012AE037ED43E25CE306D7E9
:1007500087FF0CC020E030E0A901C301B201FED642
:1007600087FF0CC0412C512C320108C05AE0452EA5
:1007700057ED552E53E2652E5CE3752E043D1E4F5A
:100780001CF4412C512C3201B8ADBF932FA92F93EB
:100790003EA93F938DA98F9320E030E040E251E4E1
:1007A000C501B4010E94410C45D77F936F9320E0AF
:1007B00030E040E251E4C701B6010E94410C3AD753
:1007C0007F936F93ABE1B1E0BF93AF93A9E2B1E048
:1007D000BF93AF930E94ED0C0FB6F894DEBF0FBE2F
:1007E000CDBF212C312C01C01C0180E091E026D529
:1007F0007FD45ECE0895089580E091E095C480E0B6
:1008000091E084C50895292F33272230310559F00E
:100810002330310569F021303105F9F482E190E0AF
:1008200026E231E01EC08EE390E028EE30E019C0F1
:1008300099278130910541F08230910541F0892B53
:1008400061F4E4EEF0E005C0EAECF0E002C0ECEAAE
:10085000F0E0849190E09F0104C080E090E020E00F
:1008600030E0FA01318320830895209142013091D4
:1008700043012617370748F06115710539F42091B7
:10088000E8002E772093E80001C0B901FC0120E0C8
:1008900061157105B9F180913B01882309F440C0CD
:1008A000853009F43FC08091E80083FD3DC0809110
:1008B000E80082FF06C08091E80082FF26C080E049
:1008C00008958091E80080FFE3CF2091F3008091AC
:1008D000F20090E0922B6115710551F0883091057E
:1008E00038F421912093F100615071090196F3CF02
:1008F00021E0089709F020E08091E8008E7780934E
:10090000E800C6CF2111C7CFD6CF80913B01882305
:1009100039F0853039F08091E80083FFCCCF04C0F6
:1009200082E0089583E0089581E0089520914201D6
:10093000309143012617370748F06115710539F4E6
:100940002091E8002E772093E80001C0B901FC0156
:1009500020E061157105C1F180913B01882309F404
:1009600041C0853009F440C08091E80083FD3EC05D
:100970008091E80082FF06C08091E80082FF27C0D6
:1009800080E008958091E80080FFE3CF2091F3009C
:100990008091F20090E0922B6115710559F088303A
:1009A000910540F424912093F10031966150710932
:1009B0000196F2CF21E0089709F020E08091E8004D
:1009C0008E778093E800C5CF2111C6CFD5CF809117
:1009D0003B01882339F0853039F08091E80083FFAE
:1009E000CBCF04C082E0089583E0089581E00895AC
:1009F000982F973058F59093E900981739F0709137
:100A0000EC002091ED005091F00003C0242F762FD0
:100A100050E021FF19C03091EB003E7F3093EB0096
:100A20003091ED003D7F3093ED003091EB0031606F
:100A30003093EB007093EC002093ED005093F000A6
:100A40002091EE0027FF07C09F5FD3CF8F70809368
:100A5000E90081E0089580E008950F931F93CF93FC
:100A6000DF93062FEC0110E0101771F198819923A4
:100A700041F12C81E981FA817B81892F8F70873048
:100A800010F080E022C0223010F056E001C052E0A9
:100A900028E030E040E02E173F0720F44F5F220FA0
:100AA000331FF9CF4295407F452B692F661F66277C
:100AB000661F90E4799F90011124622B99DF8823AF
:100AC00001F31F5F2596D0CF81E0DF91CF911F9179
:100AD0000F91089580913C0187FD05C08091E80049
:100AE00080FF0EC012C08091E80082FD05C0809199
:100AF0003B018111F8CF08958091E8008B7708C001
:100B000080913B018111EACF08958091E8008E77B2
:100B10008093E80008958091E4009091E50045E617
:100B20002091EC0020FF21C02091E80020FD21C091
:100B300020913B01222389F0253089F02091EB00A0
:100B400025FD0FC02091E4003091E50028173907FA
:100B500039F3415041F0C901E3CF82E0089583E0C9
:100B6000089581E0089584E008952091E80022FF2F
:100B7000DFCF80E008950F931F93CF93DF934BD087
:100B800052D0C8EDD0E088818F77888388818068D3
:100B9000888388818F7D888319BC10923B011092D5
:100BA0003701109239011092380100EE10E0F8017F
:100BB00080818B7F808388818160888342E060E0D0
:100BC00080E016DFE1EEF0E080818E7F8083E2EE50
:100BD000F0E0808181608083808188608083F8017B
:100BE00080818E7F8083888180618883DF91CF912F
:100BF0001F910F910895E8EDF0E080818F7E808352
:100C0000E7EDF0E080818160808384E082BF81E055
:100C100080933A01B0CFE8EDF0E080818E7F808351
:100C20001092E20008951092DA001092E100089507
:100C30001F920F920FB60F9211242F933F934F9351
:100C40005F936F937F938F939F93AF93BF93EF9334
:100C5000FF938091E10082FF0AC08091E20082FF51
:100C600006C08091E1008B7F8093E10040D28091AB
:100C7000DA0080FF1DC08091D80080FF19C08091EC
:100C8000DA008E7F8093DA008091D90080FF0CC05B
:100C900080E189BD82E189BD09B400FEFDCF81E01C
:100CA00080933B01A7DD04C019BC10923B01A3DD7A
:100CB0008091E10080FF18C08091E20080FF14C0A5
:100CC0008091E2008E7F8093E2008091E20080615B
:100CD0008093E2008091D80080628093D80019BC94
:100CE00085E080933B0103D28091E10084FF2FC017
:100CF0008091E20084FF2BC080E189BD82E189BD43
:100D000009B400FEFDCF8091D8008F7D8093D8007C
:100D10008091E1008F7E8093E1008091E2008F7EE0
:100D20008093E2008091E20081608093E2008091F4
:100D30003701882311F084E007C08091E30087FF2A
:100D400002C083E001C081E080933B01D0D180915B
:100D5000E10083FF27C08091E20083FF23C08091E0
:100D6000E100877F8093E10082E080933B01109255
:100D700037018091E1008E7F8093E1008091E20055
:100D80008E7F8093E2008091E20080618093E20098
:100D900042E060E080E02CDE8091F000886080938B
:100DA000F000A5D1FF91EF91BF91AF919F918F91ED
:100DB0007F916F915F914F913F912F910F900FBE57
:100DC0000F901F9018951F920F920FB60F9211243B
:100DD0002F933F934F935F936F937F938F939F9343
:100DE000AF93BF93CF93EF93FF93C091E900CF7080
:100DF0008091EC001092E9008091F000877F809351
:100E0000F00078941BD01092E9008091F000886087
:100E10008093F000C093E900FF91EF91CF91BF91D3
:100E2000AF919F918F917F916F915F914F913F9182
:100E30002F910F900FBE0F901F9018951F93CF9377
:100E4000DF93CDB7DEB7AA970FB6F894DEBF0FBE1B
:100E5000CDBFECE3F1E08091F100819321E0E43437
:100E6000F207C9F7CCDC8091E80083FF28C190919C
:100E70003C0180913D01853009F481C030F481301E
:100E8000A9F168F0833091F11AC1883009F4ECC0FF
:100E9000893009F4F8C0863009F011C192C0903849
:100EA00021F0923809F00BC108C08091380190916F
:100EB0003901992389F082600FC0809140018F70C1
:100EC000873008F0FCC08093E9008091EB0085FB3F
:100ED000882780F91092E9009091E800977F90931D
:100EE000E8008093F1001092F100C9C0292F2D7FF6
:100EF00009F0E5C0992319F0923061F0E0C09091BB
:100F00003E01913009F0DBC0833009F090E090930E
:100F100039012CC090913E01911128C020914001CF
:100F20002F709FEF920F963008F0C9C02093E90010
:100F30009091EB0090FF1AC0833021F48091EB0078
:100F4000806212C08091EB0080618093EB0081E0B1
:100F500090E001C0880F2A95EAF78093EA0010928A
:100F6000EA008091EB0088608093EB001092E9002A
:100F70008091E800877F8093E800ACDDA0C09111EC
:100F80009EC010913E011F778091E3008078812BF5
:100F90008093E3008091E800877F8093E8009ADDEA
:100FA0008091E80080FFFCCF8091E300806880930F
:100FB000E300112311F083E001C082E080933B0144
:100FC0007EC09058923008F07AC080913E01909196
:100FD0003F018C3D23E0920771F583E08A838AE22A
:100FE00089834FB7F894DE01139620E03EE051E28A
:100FF000E32FF0E050935700E49120FF03C0E29507
:10100000EF703F5FEF708E2F90E0EA3010F0C796E0
:1010100001C0C0968D939D932F5F243149F74FBF38
:101020008091E800877F8093E8006AE270E0CE015B
:1010300001961BDC13C06091400170914101AE012B
:101040004F5F5F4FE0DB0097D1F12091E800277FF1
:101050002093E800BC0189819A8168DC8091E800D6
:101060008B778093E8002BC0903849F58091E80099
:10107000877F8093E800809137018093F100809111
:10108000E8008E7778CF91111AC090913E0192308E
:10109000B0F48091E800877F8093E8009093370157
:1010A00019DD80913701811104C08091E30087FF31
:1010B00002C084E001C081E080933B019DDB809110
:1010C000E80083FF0AC08091E800877F8093E800F2
:1010D0008091EB0080628093EB00AA960FB6F894A3
:1010E000DEBF0FBECDBFDF91CF911F910895089550
:1010F000CF9380913B018823A9F08091E9008F7004
:101100009091EC0090FF02C090E801C090E0C92FE0
:10111000C82B1092E9008091E80083FD8FDECF702C
:10112000C093E900CF910895CF93DF93EC01FC01C8
:1011300070968BE0DF011D928A95E9F782E08C833F
:10114000898783E08E8761E0CE01019686DC882363
:1011500061F061E0CE01069680DC882331F061E029
:10116000CE010B96DF91CF9178CC80E0DF91CF91CB
:101170000895CF93C62F20913B012430F1F4FC0158
:101180004489558966897789452B462B472BA9F0D9
:1011900081818F708093E9008091E80085FF04C011
:1011A000C093F10080E00AC08091E8008E778093C0
:1011B000E800B1DC8823A1F301C082E0CF9108955B
:1011C000FB01682F84859585D4DF21E030E0811113
:1011D00002C020E030E088279927821B930B0895F6
:1011E00020913B01243041F5FC01448955896689F1
:1011F0007789452B462B472BF9F081818F7080939F
:10120000E9002091F3008091F20090E0922B892B6D
:1012100089F09091E8008091E8008E778093E80053
:1012200095FD08C078DC811108C08091E8008E77B8
:101230008093E80080E0089582E0089520913B01CA
:10124000243089F4FC014489558966897789452BC6
:10125000462B472B41F021812F702093E9002091EC
:10126000E80020FDBDCF089520913B01243019F006
:101270008FEF9FEF0895FC0144895589668977892E
:10128000452B462B472BA1F386818F708093E90075
:101290008091E80082FFECCF2091F3008091F20072
:1012A00090E0922B892B21F02091F10030E002C0D8
:1012B0002FEF3FEF4091F3008091F20090E0942BEC
:1012C000892B29F48091E8008B778093E800C9018D
:1012D0000895FC0184859585C7DF97FF02C08EEFD6
:1012E0009FEF0895FB012EE0DB011D922A95E9F79F
:1012F00023E0238320EE38E03187208729E639E098
:10130000338722879587848708950895CF93DF9345
:10131000EC018091E80083FFA6C0888190E02091D5
:101320004001309141012817390709F09CC0809194
:101330003D01813261F020F4803209F43EC093C057
:10134000823209F46CC0833209F47DC08CC0809174
:101350003C01813A09F087C08091E800877F809343
:10136000E8008091E80080FFFCCF4C895D896E89A0
:101370007F894093F100BB27A72F962F852F80935D
:10138000F100CB01AA27BB278093F100472F5527F7
:10139000662777274093F100888D8093F100898D2F
:1013A0008093F1008A8D8093F1008091E8008E7720
:1013B0008093E800DF91CF918DCB80913C01813209
:1013C00009F051C08091E800877F8093E800809108
:1013D000E80082FD05C080913B018111F8CF43C038
:1013E0003091F1002091F1009091F1008091F10095
:1013F0003C8B2D8B9E8B8F8B8091F100888F809101
:10140000F100898F8091F1008A8F8091E8008B77BD
:101410008093E8005FDBCE01DF91CF9176CF8091A2
:101420003C01813201F58091E800877F8093E800DC
:1014300051DB80913E0190913F01998B888BCE01C9
:10144000DF91CF91DFC980913C01813261F48091BD
:10145000E800877F8093E8003DDB60913E01CE018C
:10146000DF91CF9152CFDF91CF9108955058BB2794
:10147000AA270ED0B1C1A2D130F0A7D120F031F40B
:101480009F3F11F41EF497C10EF4E095E7FB64C191
:10149000E92FB3D180F3BA17620773078407950762
:1014A00018F071F49EF5E2C10EF4E0950B2EBA2F00
:1014B000A02D0B01B90190010C01CA01A00111245A
:1014C000FF27591B99F0593F50F4503E68F11A1606
:1014D000F040A22F232F342F4427585FF3CF469597
:1014E00037952795A795F0405395C9F77EF41F16B9
:1014F000BA0B620B730B840BBAF09150A1F0FF0F83
:10150000BB1F661F771F881FC2F70EC0BA0F621F6E
:10151000731F841F48F4879577956795B795F7955E
:101520009E3F08F0B3CF9395880F08F09927EE0FF0
:1015300097958795089583D180F09F3740F4911156
:101540000EF495C160E070E080E89FE3089526F016
:101550001B16611D711D811D05C11FC1D9D008F465
:1015600081E008950CD038C130D140F027D130F05F
:1015700021F45F3F19F0F0C0511179C11CC13DD178
:1015800098F39923C9F35523B1F3951B550BBB274A
:10159000AA2762177307840738F09F5F5F4F220FF7
:1015A000331F441FAA1FA9F333D00E2E3AF0E0E8F0
:1015B00030D091505040E695001CCAF729D0FE2F3C
:1015C00027D0660F771F881FBB1F261737074807CE
:1015D000AB07B0E809F0BB0B802DBF01FF27935884
:1015E0005F4F2AF09E3F510568F0B6C040C15F3F93
:1015F000ECF3983EDCF3869577956795B795F7956C
:101600009F5FC9F7880F911D9695879597F9089563
:10161000E1E0660F771F881FBB1F621773078407FF
:10162000BA0720F0621B730B840BBA0BEE1F88F70E
:10163000E095089504D06894B11119C10895E5D0DA
:1016400088F09F5790F0B92F9927B751A0F0D1F0AB
:10165000660F771F881F991F1AF0BA95C9F712C035
:10166000B13081F003D1B1E0089500C1672F782F28
:101670008827B85F39F0B93FCCF3869577956795A1
:10168000B395D9F73EF490958095709561957F4F0D
:101690008F4F9F4F0895E89409C097FB3EF49095B3
:1016A0008095709561957F4F8F4F9F4F9923A9F03B
:1016B000F92F96E9BB279395F695879577956795CA
:1016C000B795F111F8CFFAF4BB0F11F460FF1BC00E
:1016D0006F5F7F4F8F4F9F4F16C0882311F096E9A1
:1016E00011C0772321F09EE8872F762F05C066234F
:1016F00071F096E8862F70E060E02AF09A95660F08
:10170000771F881FDAF7880F9695879597F90895C0
:10171000990F0008550FAA0BE0E8FEEF1616170602
:10172000E807F907C0F012161306E407F50798F06A
:10173000621B730B840B950B39F40A2661F0232B83
:10174000242B252B21F408950A2609F4A140A695FF
:101750008FEF811D811D089597F99F6780E870E0E4
:1017600060E00895882371F4772321F09850872B47
:10177000762F07C0662311F499270DC09051862B50
:1017800070E060E02AF09A95660F771F881FDAF7FD
:10179000880F9695879597F908959F3F31F091505E
:1017A00020F4879577956795B795880F911D969545
:1017B000879597F908959FEF80EC089500240A9487
:1017C0001616170618060906089500240A9412161C
:1017D0001306140605060895092E0394000C11F44F
:1017E000882352F0BB0F40F4BF2B11F460FF04C0FC
:1017F0006F5F7F4F8F4F9F4F089557FD9058440F55
:10180000551F59F05F3F71F04795880F97FB991F5F
:1018100061F09F3F79F0879508951216130614061C
:10182000551FF2CF4695F1DF08C0161617061806A9
:10183000991FF1CF86957105610508940895E5DF3C
:10184000A0F0BEE7B91788F4BB279F3860F41616DE
:10185000B11D672F782F8827985FF7CF86957795EA
:101860006795B11D93959639C8F30895E894BB2701
:1018700066277727CB0197F908954ADF08F48FEFA1
:1018800008950BD0A9CF9ADF28F09FDF18F0952399
:1018900009F062CF90CF1124EACFAFDFA0F3959F7C
:1018A000D1F3950F50E0551F629FF001729FBB2747
:1018B000F00DB11D639FAA27F00DB11DAA1F649FF3
:1018C0006627B00DA11D661F829F2227B00DA11DA6
:1018D000621F739FB00DA11D621F839FA00D611D2C
:1018E000221F749F3327A00D611D231F849F600D4D
:1018F000211D822F762F6A2F11249F5750408AF086
:10190000E1F088234AF0EE0FFF1FBB1F661F771F11
:10191000881F91505040A9F79E3F510570F01CCF91
:10192000A6CF5F3FECF3983EDCF3869577956795FD
:10193000B795F795E7959F5FC1F7FE2B880F911D2F
:101940009695879597F9089511F40EF434CF25CF25
:101950005CDFD0F39923D9F3CEF39F57550B87FF64
:1019600035D00024A0E640EA90018058569597951E
:1019700028F4805C660F771F881F20F02617370732
:10198000480730F4621B730B840B202931294A2B42
:10199000A69517940794202531254A2758F7660FF6
:1019A000771F881F20F026173707480730F4620B8F
:1019B000730B840B200D311D411DA09581F7B901DA
:1019C000842F9158880F969587950895915050408F
:1019D000660F771F881FD2F70895A0E0B0E0E2EF0E
:1019E000FCE083C2AE01475F5F4F6F8178858D81D8
:1019F0009E8102D0E2E095C2ACE0B0E0E1E0FDE023
:101A000064C27C016B018A01FC011782168283810A
:101A100081FFB0C1CE0101964C01F7019381F6011F
:101A200093FD859193FF81916F01882309F49EC1F5
:101A3000853239F493FD859193FF81916F01853251
:101A400021F4B70190E0B1D1E8CF512C312C20E046
:101A50002032A0F48B3269F030F4803259F08332B6
:101A600069F420612CC08D3239F0803339F4216063
:101A700026C02260246023C0286021C027FD27C023
:101A800030ED380F3A3078F426FF06C0FAE05F9E5A
:101A9000300D1124532E13C08AE0389E300D1124CE
:101AA000332E20620CC08E3221F426FD5FC12064EB
:101AB00006C08C3611F4206802C0883641F4F60165
:101AC00093FD859193FF81916F018111C1CF982F73
:101AD0009F7D9554933028F40C5F1F4FFFE3F983EB
:101AE0000DC0833631F0833771F0833509F057C06C
:101AF00021C0F801808189830E5F1F4F44244394E5
:101B0000512C540114C03801F2E06F0E711CF80121
:101B1000A080B18026FF03C0652D70E002C06FEF8A
:101B20007FEFC5012C8736D12C0183012C852F77BF
:101B3000222E16C03801F2E06F0E711CF801A08051
:101B4000B18026FF03C0652D70E002C06FEF7FEF0C
:101B5000C5012C8714D12C012C852068222E8301ED
:101B600023FC19C0832D90E048165906A0F4B70154
:101B700080E290E01AD13A94F5CFF50127FC8591E7
:101B800027FE81915F01B70190E00FD131103A94A7
:101B9000F1E04F1A51084114510479F7DEC0843640
:101BA00011F0893631F5F80127FF07C06081718196
:101BB000828193810C5F1F4F08C0608171818827EB
:101BC00077FD8095982F0E5F1F4F2F76B22E97FFCF
:101BD00009C090958095709561957F4F8F4F9F4F6D
:101BE0002068B22E2AE030E0A40111D1A82EA81856
:101BF00043C0853729F42F7EB22E2AE030E025C07D
:101C0000F22FF97FBF2E8F36C1F018F4883579F0A6
:101C1000ADC0803719F0883721F0A8C02F2F206180
:101C2000B22EB4FE0DC08B2D8460B82E09C024FFE7
:101C30000AC09F2F9660B92E06C028E030E005C08C
:101C400020E130E002C020E132E0F801B7FE07C039
:101C500060817181828193810C5F1F4F06C060811A
:101C6000718180E090E00E5F1F4FA401D0D0A82EBC
:101C7000A818FB2DFF77BF2EB6FE0BC02B2D2E7F95
:101C8000A51450F4B4FE0AC0B2FC08C02B2D2E7E61
:101C900005C07A2C2B2D03C07A2C01C0752C24FF93
:101CA0000DC0FE01EA0DF11D8081803311F4297E03
:101CB00009C022FF06C07394739404C0822F8678F3
:101CC00009F0739423FD12C020FF06C05A2C731430
:101CD00018F4530C5718732C731460F4B70180E296
:101CE00090E02C8762D073942C85F6CF731410F497
:101CF000371801C0312C24FF11C0B70180E390E0F8
:101D00002C8753D02C8522FF16C021FF03C088E505
:101D100090E002C088E790E0B7010CC0822F86787F
:101D200051F021FD02C080E201C08BE227FD8DE26F
:101D3000B70190E03AD0A51430F4B70180E390E009
:101D400034D05A94F8CFAA94F401EA0DF11D8081A1
:101D5000B70190E02AD0A110F6CF332009F45DCE70
:101D6000B70180E290E021D03A94F7CFF701868165
:101D7000978102C08FEF9FEF2C96E2E1C2C0FC0179
:101D80000590615070400110D8F7809590958E0FA6
:101D90009F1F0895FC016150704001900110D8F719
:101DA000809590958E0F9F1F08950F931F93CF934B
:101DB000DF93182F092FEB018B8181FD03C08FEF7B
:101DC0009FEF20C082FF10C04E815F812C813D813A
:101DD000421753077CF4E881F9819F012F5F3F4F41
:101DE00039832883108306C0E885F985812F0995FA
:101DF000892B29F72E813F812F5F3F4F3F832E8311
:101E0000812F902FDF91CF911F910F910895FA01AB
:101E1000AA27283051F1203181F1E8946F936E7F29
:101E20006E5F7F4F8F4F9F4FAF4FB1E03ED0B4E01A
:101E30003CD0670F781F891F9A1FA11D680F791F5B
:101E40008A1F911DA11D6A0F711D811D911DA11D6C
:101E500020D009F468943F912AE0269F112430197C
:101E6000305D3193DEF6CF010895462F4770405D17
:101E70004193B3E00FD0C9F7F6CF462F4F70405DC6
:101E80004A3318F0495D31FD4052419302D0A9F721
:101E9000EACFB4E0A6959795879577956795BA951B
:101EA000C9F700976105710508959B01AC010A2EE1
:101EB00006945795479537952795BA95C9F7620FB8
:101EC000731F841F951FA01D08952F923F924F925C
:101ED0005F926F927F928F929F92AF92BF92CF92BA
:101EE000DF92EF92FF920F931F93CF93DF93CDB7C3
:101EF000DEB7CA1BDB0B0FB6F894DEBF0FBECDBF3B
:101F000009942A88398848885F846E847D848C840B
:101F10009B84AA84B984C884DF80EE80FD800C8114
:101F20001B81AA81B981CE0FD11D0FB6F894DEBFF7
:0C1F30000FBECDBFED010895F894FFCF67
:101F3C000083100000010410000001820800000161
:101F4C000000000000000000000000256420256453
:081F5C002025642025640A0021
:00000001FF
